:100000008A110A1205280000090007309F00831694
:1000100086010130850083120614F430A0000130FF
:10002000A1008A231822EC223120AC012C08053CC7
:10003000031C2D28AD012D083B3C031C2728023052
:10004000A000A1018A230130AD07031C1B281F302B
:1000500083050130AC07031C16281F3083050C28CC
:100060003028061086178616F430A0000130A10053
:100070008A2389208920962096209620892089200D
:10008000AD012D08033C031C5128A720AF20B72049
:10009000BF20C720BF20892089200130AD07031C65
:1000A00041281F308305CF20892096209620962056
:1000B00089208920D7208920D7208920D72089200E
:1000C0008920AD012D08023C031C7728E1208920FE
:1000D000EB208920F3208920052189200E21892009
:1000E0000521892089200130AD07031C62281F30BB
:1000F00083051A2189209030A0000130A1008A23B5
:100100008613861206142C30A0000130A1008A2329
:100110000800AC012C08063C031C93282421013064
:10012000AC07031C8A281F3083050800AC012C088B
:10013000023C031CA02824210130AC07031C972893
:100140001F308305CB21CB21242124210800242129
:100150003E21CB21CB21CB21CB21242108002421FE
:10016000DA21BB21CB21BB21DA2124210800242163
:100170009A21EA21EA21EA21DA2124210800242116
:100180004D213E214D214D21AA2124210800242169
:100190004D213E21EA21F221802124210800242141
:1001A0004D213E21EA215E214D21242108003121EB
:1001B00024213121242131212421312131213121D6
:1001C0000800312124213121312131212421312103
:1001D0002421312108003121242131212421312100
:1001E00031213121080031213121312124213121D6
:1001F0003121312124213121312131212421312189
:1002000031213121242131210800242131213121C2
:1002100031212421312124213121080031212421BF
:100220003121312131212421312131213121242158
:100230003121080031213121312124213121242192
:100240003121312131210800AE012E08063C031C6A
:100250002E2903220130AE07031C25291F308305F8
:100260000800AE012E08063C031C3B290922013080
:10027000AE07031C32291F30830508000322AE019C
:100280002E08043C031C492909220130AE07031C37
:1002900040291F3083050322080003220922AE01F2
:1002A0002E08023C031C592903220130AE07031C0F
:1002B00050291F308305092203220800032203224C
:1002C000092203220922032203220800AE012E087C
:1002D000023C031C702903220130AE07031C67296E
:1002E0001F3083050922AE012E08023C031C7D2924
:1002F00003220130AE07031C74291F308305080058
:10030000AE012E08023C031C8A2903220130AE07ED
:10031000031C81291F308305AE012E08023C031CFB
:10032000962909220130AE07031C8D291F30830551
:1003300003220800AE012E08033C031CA42903225B
:100340000130AE07031C9B291F30830509220922B7
:100350000322080003220322AE012E08023C031CE4
:10036000B62909220130AE07031CAD291F308305D1
:10037000032203220800032203220922AE012E08D1
:10038000033C031CC82903220130AE07031CBF290C
:100390001F308305080003220922AE012E08043C09
:1003A000031CD72903220130AE07031CCE291F30BE
:1003B0008305080003220322AE012E08033C031C20
:1003C000E62909220130AE07031CDD291F30830511
:1003D0000322080003220922032209220322092200
:1003E00003220800AE012E08023C031CFC29032254
:1003F0000130AE07031CF3291F30830509220322B5
:1004000009220322080086110830A000A1018A23D6
:1004100008008615063084001030AA00FD30A000C8
:100420000130A1000830A2000030A300C52308005D
:10043000061086178616F430A0000130A1008A232A
:10044000B122612261226A2261226122AC012C0860
:10045000023C031C432A84229F22BA22C322B122D7
:1004600072228D227222AD012D08023C031C3D2A0E
:1004700058220130AD07031C342A1F308305013098
:10048000AC07031C272A1F3083057B2261226122CF
:10049000612261229030A0000130A1008A238613DE
:1004A000861206142C30A0000130A1008A23080017
:1004B000DC22DC22DC22CC22DC22DC22CC22CC227C
:1004C0000800DC22DC22DC22DC22CC22DC22CC2252
:1004D000CC2208009622A8229622A8229622A822A0
:1004E00096220800DC22CC22DC22DC22CC22DC2278
:1004F000CC22CC220800DC22CC22CC22CC22CC2262
:10050000DC22CC22CC220800DC22DC22CC22DC2221
:10051000DC22CC22CC22CC220800DC22DC22CC2221
:10052000CC22DC22CC22CC22CC220800DC22DC2211
:10053000CC22DC22CC22DC22CC22CC220800DC2201
:10054000CC22CC22CC22DC22DC22CC22CC22080001
:10055000DC22CC22DC22CC22DC22CC22CC22CC22FB
:100560000800DC22CC22CC22CC22CC22CC22CC22F1
:10057000CC220800DC22CC22CC22DC22CC22CC22D1
:10058000CC22CC220800DC22DC22DC22DC22CC22A1
:10059000CC22CC22CC2208008615063084001030F4
:1005A000AA005730A0000130A1002030A200003086
:1005B000A300C5238611080086150630840010307C
:1005C000AA008730A0000130A1001C30A20000303A
:1005D000A300C52386110800061086178616F4307E
:1005E000A0000130A1008A2321233F2321233F23A0
:1005F00021234D232C232C230F239030A0000130E6
:10060000A1008A238613861206142C30A000013024
:10061000A1008A230800762363236323080076233E
:100620006323762308006323762363236323080070
:1006300063237623762363230800632363237623CF
:10064000080063236323632376230800762376233D
:10065000762376236323080013233F231D233F23A0
:1006600026233F230B233F2318233F230B234D2314
:10067000080086113C30A000A1018A2308008611E1
:100680003C30A000A1018A233C30A000A1018A23B4
:100690003C30A000A1018A23080086113C30A00054
:1006A000A1018A233C30A000A1018A233C30A00094
:1006B000A1018A233C30A000A1018A233C30A00084
:1006C000A1018A2308008615061506308400103023
:1006D000AA00F330A0000130A1003C30A20000309D
:1006E000A300C523861106113923080086150615B7
:1006F000063084001030AA00F330A0000130A100C1
:10070000F030A2000030A300C52386110611392362
:100710000800892BA0080319952B9C23A003000037
:1007200000000000000000008A2BA1080319080047
:100730009C23A103A0038A2B0C30A500A50B9E2BA4
:10074000000000001230A200A20BAB2BAD23AD23A2
:10075000000000000800AD23A42B0D30A400A40B62
:10076000AF2B000008001030A8020001031C013E5E
:10077000A902031C0800BC2B0A30A8020001031CBC
:10078000013EA902031C0800BC2B2A088004200893
:10079000A8002108A900B3230130A202031CA3036F
:1007A0002A0980052008A8002108A900B323A2086F
:0C07B000031DC52BA308031DC52B08006A
:02400E00F13F80
:00000001FF
